:020000040000FA
:0A000000000000008FEF00F09DD01B
:08001800EAD00E6E960E056E93
:10002000980E066E55D8D8B4CA90D8A4CA80FC0FD2
:10003000D8A0CA92D8B0CA82800E056E960E066EFF
:10004000980E096E0A6ACAB025D8CAB223D842D817
:100050000504CB6E05C007F006C008F000500B6E1B
:100060000C6E003C0C6A4BD80A500E2E0AD0BE6EA5
:100070000C0EBD6E09BEBD8A09BCBD889394CA84AE
:100080001200BB6E0C0EBA6E09BEBA8A09BCBA88E1
:100090009492F5D700D8D890093206320532120072
:1000A000086A076EFF0E0726082200D0D8A01200AB
:1000B000030E066EE60E02D8F5D7066AFE0F056E31
:1000C000E86A065AD8A012000000050600D0F8D74A
:1000D0000A6A096A100EF36E063409360A360750AA
:1000E000095C08500A5805E30750095E08500A5A8F
:1000F000D88005360636F32EEFD70550120007508C
:100100000B02F3CF09F0F4CF0AF008500B02F350C2
:100110000A2607500C02F3500A26095012004F0E0F
:10012000AF6E240EAC6E900EAB6E0001C69A430EFD
:10013000926EE00E936EC00E946E0F0EC16E070E9F
:10014000B46E6CD0F2A403D0F294817A11009EAA0E
:1001500019D0060EAB1412E1E2CF4AF0E1CF49F01C
:100160004B2A11EE00F04B50E126000EE222AECFFA
:10017000E7FF4AC0E2FF49C0E1FF1100AE50AE50B8
:10018000AB98AB8811004B504C5C14E04C2AEACF82
:1001900006F0E9CF05F001EE00F04C50E926000E24
:1001A000EA22EF50056E06C0EAFF05C0E9FFD880DD
:1001B000120004D0E868056ED8A0120012004B6A45
:1001C0004C6A9D8A9F8AF28EF28C12009D9A01EEF3
:1001D00000F0010EF46EF36AF306000EF45AEE6AB4
:1001E000F450F310F9E14B6A4C6A9D8A1200F29EBA
:1001F000E0CF61F8D8CF62F8E8CF63F8F28E000163
:10020000A192F29E61C8E0FF62C8D8FF63C8E8FF10
:10021000F28E10009EA8FED7AD6E120094908B90C7
:10022000949A8B9A94988B9893908A9093928A92AE
:1002300094968B96939A8A9A92988998929A899A88
:1002400092968996256A2C6A2D6A520E236E680E44
:10025000226E200E216E206A205022242A6E215008
:1002600023202B6E1C0E2E6E006A2BC008F02AC0B5
:1002700007F0020ED2DE006A2BC008F02AC007F099
:10028000010ECBDE69EC06F0939A8A8A320E08DF03
:10029000939A8A9A246A296A92DF98DFCD6AF29447
:1002A000F28A870ED56EB16AA192A082B36AB26A51
:1002B000D08EA292B00EB16E00EE4DF0140EEE682C
:1002C000E82EFDD74868478E416A406A3F6A3E6A19
:1002D000422AE86A42B2010F43B0010806E14370C6
:1002E0003E2A000E3F22402241224DDF116EEC0ECD
:1002F000115C09E3FE0E115C03E3ADEF03F003D0E4
:10030000136AADEF03F011AE37D0136A8B0E115C98
:1003100005E111C013F0146815682DD09B0E115C17
:1003200005E111C013F01668176825D0AB0E115CFB
:1003300005E111C013F0186819681DD0BB0E115CDF
:1003400005E111C013F01A681B6815D0CB0E115CC3
:1003500004E111C013F01C680ED0DB0E115C04E147
:1003600011C013F01D6807D0EB0E115C04E111C041
:1003700013F01E681F68F0D1135202E1EED1ECD1E8
:100380008B0E135C2EE1142803E111C014F027D06A
:100390000C0E145C04E18B9A299024901ED00D0E53
:1003A000145C04E18B982992249217D00E0E145CF1
:1003B00004E1299424948A9010D00F0E145C04E177
:1003C000299624968A9209D0100E145C04E129988B
:1003D00024988B9602D01468C0D11468BDD1BDD1C9
:1003E000BBD19B0E135CD8A415D1162803E111C014
:1003F00016F00ED111C017F0175227E10C0E165C43
:1004000004E18B9A299024901ED00D0E165C04E115
:100410008B982992249217D00E0E165C04E1299431
:1004200024948A9010D00F0E165C04E1299624962D
:100430008A9209D0100E165C04E1299824988B96B4
:1004400002D016688AD1166887D12552D8B4E0D078
:100450000C0E165C29E18B8A7F0E175C22E207EEF8
:1004600061F0D8901734E926000EEA22EECF2FF083
:10047000EFCF30F024802F503E24016E30503F20CB
:10048000026E000E4020036E000E4120046E04C078
:1004900050F003C04FF002C04EF001C04DF0298073
:1004A00002D024902980B2D00D0E165C29E18B88F1
:1004B0007F0E175C22E207EE61F0D8901734E92630
:1004C000000EEA22EECF31F0EFCF32F0248231502D
:1004D0003E24016E32503F20026E000E4020036E1B
:1004E000000E4120046E04C054F003C053F002C05B
:1004F00052F001C051F0298202D02492298286D084
:100500000E0E165C29E18A807F0E175C22E207EE50
:1005100061F0D8901734E926000EEA22EECF33F0CE
:10052000EFCF34F0248433503E24016E34503F200A
:10053000026E000E4020036E000E4120046E04C0C7
:1005400058F003C057F002C056F001C055F029849E
:1005500002D0249429845AD00F0E165C29E18A8295
:100560007F0E175C22E207EE61F0D8901734E9267F
:10057000000EEA22EECF35F0EFCF36F0248635506C
:100580003E24016E36503F20026E000E4020036E66
:10059000000E4120046E04C05CF003C05BF002C09A
:1005A0005AF001C059F0298602D0249629862ED00F
:1005B000100E165C29E18B867F0E175C22E207EE97
:1005C00061F0D8901734E926000EEA22EECF37F01A
:1005D000EFCF38F0248837503E24016E38503F204A
:1005E000026E000E4020036E000E4120046E04C017
:1005F00060F003C05FF002C05EF001C05DF02988CA
:1006000002D02498298802D01668A7D01668A4D0F2
:10061000A4D0A2D0AB0E135CD8A47BD0182804E1E0
:1006200011C018F09AD074D00C0E185C14E111C0EF
:1006300039F039520CE007EE61F0D8903934E926F0
:10064000000EEA22EECF2FF0EFCF30F003D0306A69
:100650002F6A29905BD00D0E185C14E111C03AF09E
:100660003A520CE007EE61F0D8903A34E926000ED9
:10067000EA22EECF31F0EFCF32F003D0326A316AA6
:10068000299244D00E0E185C14E111C03BF03B528D
:100690000CE007EE61F0D8903B34E926000EEA2228
:1006A000EECF33F0EFCF34F003D0346A336A2994BD
:1006B0002DD00F0E185C14E111C03CF03C520CE040
:1006C00007EE61F0D8903C34E926000EEA22EECF26
:1006D00035F0EFCF36F003D0366A356A299616D05A
:1006E000100E185C13E111C03DF03D520CE007EE16
:1006F00061F0D8903D34E926000EEA22EECF37F0C3
:10070000EFCF38F003D0386A376A2998186825D0B7
:1007100023D0BB0E135C0AE11A2803E111C01AF0C2
:1007200003D011C01BF05AD918D016D0CB0E135CD1
:1007300007E11C2803E111C01CF029D90ED00CD010
:10074000EB0E135C09E11E2803E111C01EF003D07B
:1007500011C01FF01ED901D0E0D8050E485CD8B0FA
:10076000D3D044503E5C45503F58465040584750C7
:100770004158D8A0AAD0478E48521FE129B007D0CF
:1007800024908B9A50684F684E684D6815D0827AD5
:100790002F503E24016E30503F20026E000E40204C
:1007A000036E000E4120046E04C050F003C04FF0F1
:1007B00002C04EF001C04DF087D0010E485C1FE131
:1007C00029B207D024928B985468536852685168B4
:1007D00015D0827831503E24016E32503F20026E97
:1007E000000E4020036E000E4120046E04C054F041
:1007F00003C053F002C052F001C051F065D0020EA8
:10080000485C1FE129B407D024948A90586857683F
:100810005668556815D0817033503E24016E3450AF
:100820003F20026E000E4020036E000E4120046E39
:1008300004C058F003C057F002C056F001C055F094
:1008400043D0030E485C1FE129B607D024968A9254
:100850005C685B685A68596815D0817235503E24CF
:10086000016E36503F20026E000E4020036E000ED7
:100870004120046E04C05CF003C05BF002C05AF07B
:1008800001C059F021D0040E485C1EE129B807D000
:1008900024988B9660685F685E685D6815D0827684
:1008A00037503E24016E38503F20026E000E40202B
:1008B000036E000E4120046E04C060F003C05FF0C0
:1008C00002C05EF001C05DF028D841AE1CD0416A84
:1008D000406A3F6A3E6A246A296A00EE4DF0140EAF
:1008E000EE68E82EFDD7006A2BC008F02AC007F09A
:1008F000010E0DEC00F0006A2BC008F02AC007F0D2
:10090000020E0DEC00F006D041AE04D0416A406A00
:100910003F6A3E6A817468EF01F04868478E126A48
:10092000050E125C33E2D8901234E96EEA6AEA36B8
:10093000E936EA364D0EE926000EEA22EFCF01F045
:10094000ECCF02F0ECCF03F0ECCF04F04450015CAC
:1009500045500258465003584750045815E2D89065
:100960001234E96EEA6AEA36E936EA364D0EE926CD
:10097000000EEA22EFCF44F0ECCF45F0ECCF46F08A
:10098000ECCF47F012C048F0122ACAE312001C68EC
:100990001200D8901F30216E206A20321E5020266F
:1009A000000E2122205022242A6E215023202B6E5B
:1009B0002DC000F02BC008F02AC007F0020E0DEC8D
:1009C00000F02CC000F02BC008F02AC007F0010E88
:1009D0000DEC00F01E6812001D681200070E1A5C74
:1009E0000DE1D8901B342C6E2CC000F02BC008F009
:1009F0002AC007F0010E0DEC00F026D1080E1A5C9B
:100A00000CE11BC02DF02DC000F02BC008F02AC057
:100A100007F0020E0DEC00F017D11E0E1A5CD8A4E0
:100A200055D01B5211E1296A306A2F6A396A326A3D
:100A3000316A3A6A346A336A3B6A366A356A3C6AB2
:100A4000386A376A3D6A41D01BC039F007EE61F061
:100A5000D8901B34E926000EEA22EECF2FF0EFCF1C
:100A600030F01BC03AF007EE61F0D8901B34E92655
:100A7000000EEA22EECF31F0EFCF32F01BC03BF098
:100A800007EE61F0D8901B34E926000EEA22EECF83
:100A900033F0EFCF34F01BC03CF007EE61F0D8909C
:100AA0001B34E926000EEA22EECF35F0EFCF36F008
:100AB0001BC03DF007EE61F0D8901B34E926000E14
:100AC000EA22EECF37F0EFCF38F0BED01F0E1A5C1F
:100AD000D8A4A8D089860C0E1B5C06E2520E236EA9
:100AE000680E226E899683D00C0E1B5C05E1200EE9
:100AF000236EB40E226E7BD00D0E1B5C05E1220E20
:100B0000236EA60E226E73D00E0E1B5C05E1240E22
:100B1000236EB50E226E6BD00F0E1B5C05E1260E08
:100B2000236EE40E226E63D0100E1B5C05E1290ECD
:100B3000236E340E226E5BD0110E1B5C05E12B0E72
:100B4000236EA70E226E53D0120E1B5C05E12E0EF3
:100B5000236E400E226E4BD0130E1B5C04E1310E4F
:100B6000236E226A44D0140E1B5C05E1330E236E03
:100B7000E90E226E3CD0150E1B5C04E1370E236E8D
:100B8000226A35D0160E1B5C05E13A0E236E450E27
:100B9000226E2DD0170E1B5C05E13D0E236EBC0EA0
:100BA000226E25D0180E1B5C05E1410E236E680EE7
:100BB000226E1DD0190E1B5C05E1450E236E4B0EF7
:100BC000226E15D01A0E1B5C05E1490E236E6A0ECB
:100BD000226E0DD01B0E1B5C05E14D0E236EC80E60
:100BE000226E05D0520E236E680E226E899620501A
:100BF00022242A6E215023202B6E1BC02EF02DC0E4
:100C000000F02BC008F02AC007F0020E0DEC00F037
:100C10002CC000F02BC008F02AC007F0010E0DEC2C
:100C200000F012D0420E1A5C0BE11B5205E18B90D2
:100C300025D88998256A03D08B808988256804D0B7
:100C40007B0E1A5CD8B402D81A681200246A006AB3
:100C50002BC008F02AC007F0010E0DEC00F0006A6E
:100C60002BC008F02AC007F0020E0DEC00F08B9AA2
:100C70008B98296A8A908A928B96120094908B9016
:100C8000246A8A908A928B96296A8B9A8B982C6A0E
:100C90002D6A2E6A520E236E680E226E200E216E71
:100CA000206A205022242A6E215023202B6E006AB5
:100CB0002BC008F02AC007F0010E0DEC00F0006A0E
:100CC0002BC008F02AC007F0020E0DEC00F0899648
:100CD0001200070162696169A20E646FC30E636F3F
:100CE0009A0E666F460E656F960E686F320E676FCE
:100CF000920E6A6F3A0E696F8E0E6C6F5D0E6B6F9F
:100D00008A0E6E6F9A0E6D6F860E706FF00E6F6F9B
:100D1000830E726F5F0E716F7F0E746FE70E736FCD
:100D20007C0E766F850E756F790E786F3B0E776F40
:100D3000760E7A6F070E796F720E7C6FE80E7B6FFE
:100D40006F0E7E6FDF0E7D6F6C0E806FEA0E7F6F11
:100D50006A0E826F0A0E816F670E846F3C0E836F7E
:100D6000640E866F820E856F610E886FDA0E876F54
:100D70005F0E8A6F440E896F5C0E8C6FBF0E8B6F97
:100D80005A0E8E6F4C0E8D6F570E906FE90E8F6F4F
:100D9000550E926F960E916F530E946F936F510E86
:100DA000966F200E956F4E0E986FFB0E976F4C0E40
:100DB0009A6FE50E996F4A0E9C6FDC0E9B6F480E82
:100DC0009E6FE20E9D6F460EA06FF50E9F6F450E53
:100DD000A26F150EA16F430EA46F420EA36F410EBA
:100DE000A66F7B0EA56F3F0EA86FC00EA76F3E0EBD
:100DF000AA6F100EA96F3C0EAC6F6D0EAB6F3A0E62
:100E0000AE6FD40EAD6F390EB06F460EAF6F370EAA
:100E1000B26FC20EB16F360EB46F490EB36F340E9F
:100E2000B66FDA0EB56F330EB86F740EB76F320E41
:100E3000BA6F180EB96F300EBC6FC50EBB6F2F0E98
:100E4000BE6F7B0EBD6F2E0EC06F3A0EBF6F2D0EA4
:100E5000C26F020EC16F2B0EC46FD10EC36F2A0E6C
:100E6000C66FA90EC56F290EC86F880EC76F280EF2
:100E7000CA6F6F0EC96F270ECC6F5E0ECB6F260E3A
:100E8000CE6F530ECD6F250ED06F500ECF6F240E48
:100E9000D26F540ED16F230ED46F5E0ED36F220E1D
:100EA000D66F6F0ED56F210ED86F860ED76F200EBE
:100EB000DA6FA30ED96F1F0EDC6FC60EDB6F1E0E2E
:100EC000DE6FEF0EDD6F1E0EE06FDF6F1D0EE26F47
:100ED000520EE16F1C0EE46F8C0EE36F1B0EE66F7B
:100EE000CB0EE56F1B0EE86F0F0EE76F1A0EEA6F61
:100EF000580EE96F190EEC6FA50EEB6F180EEE6F22
:100F0000F80EED6F180EF06F4F0EEF6F170EF26FB9
:100F1000AB0EF16F170EF46F0A0EF36F160EF66F2D
:100F20006F0EF56F150EF86FD70EF76F150EFA6F7F
:100F3000430EF96F140EFC6FB30EFB6F140EFE6FB1
:100F4000270EFD6F130E0801006F9F0E0701FF6F44
:100F5000130E0801026F1A0E016F120E046F990E24
:100F6000036F120E066F1B0E056F110E086FA10E98
:100F7000076F110E0A6F290E096F100E0C6FB50E58
:100F80000B6F100E0E6F440E0D6F0F0E106FD60EFE
:100F90000F6F0F0E126F6B0E116F0F0E146F030E8B
:100FA000136F0E0E166F9D0E156F0E0E186F3A0E04
:100FB000176F0D0E1A6FDA0E196F0D0E1C6F7C0E67
:100FC0001B6F0D0E1E6F210E1D6F0C0E206FC80EB5
:100FD0001F6F0C0E226F720E216F0C0E246F1E0EEF
:100FE000236F0B0E266FCC0E256F0B0E286F7C0E19
:100FF000276F0B0E2A6F2E0E296F0A0E2C6FE30E31
:101000002B6F0A0E2E6F990E2D6F0A0E306F510E38
:101010002F6F0A0E326F0B0E316F090E346FC80E30
:10102000336F090E366F850E356F090E386F450E1A
:10103000376F090E3A6F060E396F080E3C6FC90EF6
:101040003B6F080E3E6F8E0E3D6F080E406F540EC4
:101050003F6F080E426F1C0E416F070E446FE50E86
:10106000436F070E466FAF0E456F070E486F7B0E3E
:10107000476F070E4A6F490E496F070E4C6F170EE8
:101080004B6F060E4E6FE70E4D6F060E506FB90E8A
:101090004F6F060E526F8B0E516F060E546F5F0E20
:1010A000536F060E566F340E556F060E586F0A0EAC
:1010B000576F050E5A6FE10E596F050E5C6FB90E32
:1010C0005B6F050E5E6F930E5D6F050E606F6D0EAC
:1010D0005F6F000112000201646BB80E636F666BF4
:1010E000BA0E656F686BBB0E676F6A6BBC0E696F7B
:1010F0006C6BBD0E6B6F6E6BBE0E6D6F706BBF0E4B
:101100006F6F726BC10E716F746BC20E736F766B03
:10111000C30E756F786BC40E776F7A6BC50E796FDF
:101120007C6BC60E7B6F7E6BC80E7D6F806BC90EAD
:101130007F6F826BCA0E816F846BCB0E836F866B61
:10114000CC0E856F886BCD0E876F8A6BCF0E896F43
:101150008C6BD00E8B6F8E6BD10E8D6F906BD20E11
:101160008F6F926BD30E916F946BD40E936F966BBF
:10117000D60E956F986BD70E976F9A6BD80E996FA6
:101180009C6BD90E9B6F9E6BDA0E9D6FA06BDB0E76
:101190009F6FA26BDC0EA16FA46BDE0EA36FA66B1C
:1011A000DF0EA56FA86BE00EA76FAA6BE10EA96F0B
:1011B000AC6BE20EAB6FAE6BE30EAD6FB06BE50EDA
:1011C000AF6FB26BE60EB16FB46BE70EB36FB66B79
:1011D000E80EB56FB86BE90EB76FBA6BEA0EB96F70
:1011E000BC6BEC0EBB6FBE6BED0EBD6FC06BEE0E3D
:1011F000BF6FC26BEF0EC16FC46BF00EC36FC66BD7
:10120000F10EC56FC86BF30EC76FCA6BF40EC96FD2
:10121000CC6BF50ECB6FCE6BF60ECD6FD06BF70EA1
:10122000CF6FD26BF80ED16FD46BF90ED36FD66B34
:10123000FB0ED56FD86BFC0ED76FDA6BFD0ED96F36
:10124000DC6BFE0EDB6FDE6BDD69010EE06FDF6BCA
:10125000E26F020EE16F010EE46F030EE36F010E09
:10126000E66F040EE56F010EE86F050EE76F010EE5
:10127000EA6F060EE96F010EEC6F070EEB6F010EC1
:10128000EE6F090EED6F010EF06F0A0EEF6F010E9B
:10129000F26F0B0EF16F010EF46F0C0EF36F010E77
:1012A000F66F0D0EF56F010EF86F0E0EF76F010E53
:1012B000FA6F100EF96F010EFC6F110EFB6F010E2D
:1012C000FE6F120EFD6F010E0301006F130E02017F
:1012D000FF6F010E0301026F140E016F010E046F08
:1012E000150E036F010E066F170E056F010E086FC6
:1012F000180E076F010E0A6F190E096F010E0C6FA1
:101300001A0E0B6F010E0E6F1B0E0D6F010E106F7C
:101310001C0E0F6F010E126F1D0E116F010E146F58
:101320001F0E136F010E166F200E156F010E186F32
:10133000210E176F010E1A6F220E196F010E1C6F0E
:10134000230E1B6F010E1E6F240E1D6F010E206FEA
:10135000260E1F6F010E226F270E216F010E246FC4
:10136000280E236F010E266F290E256F010E286FA0
:101370002A0E276F010E2A6F2B0E296F010E2C6F7C
:101380002D0E2B6F010E2E6F2E0E2D6F010E306F56
:101390002F0E2F6F010E326F300E316F010E346F32
:1013A000310E336F010E366F320E356F010E386F0E
:1013B000340E376F010E3A6F350E396F010E3C6FE8
:1013C000360E3B6F010E3E6F370E3D6F010E406FC4
:1013D000380E3F6F010E426F390E416F010E446FA0
:1013E0003A0E436F010E466F3C0E456F010E486F7B
:1013F0003D0E476F010E4A6F3E0E496F010E4C6F56
:101400003F0E4B6F010E4E6F400E4D6F010E506F31
:10141000410E4F6F010E526F430E516F010E546F0C
:10142000440E536F010E566F450E556F010E586FE7
:10143000460E576F010E5A6F470E596F010E5C6FC3
:10144000480E5B6F010E5E6F4A0E5D6F010E606F9E
:101450004B0E5F6F646B2F0E636F666B340E656FA0
:10146000686B390E676F6A6B3E0E696F6C6B420E6C
:101470006B6F6E6B470E6D6F706B4C0E6F6F726B98
:10148000510E716F746B560E736F766B5B0E756FCA
:10149000786B600E776F7A6B650E796F7C6B690E77
:1014A0007B6F7E6B6E0E7D6F806B730E7F6F826BBA
:1014B000780E816F846B7D0E836F866B820E856FD5
:1014C000886B870E876F8A6B8C0E896F8C6B900E82
:1014D0008B6F8E6B950E8D6F906B9A0E8F6F926BDC
:1014E0009F0E916F946BA40E936F966BA90E956FE0
:1014F000986BAE0E976F9A6BB30E996F9C6BB70E8D
:101500009B6F9E6BBC0E9D6FA06BC10E9F6FA26BFD
:10151000C60EA16FA46BCB0EA36FA66BD00EA56FEA
:10152000A86BD50EA76FAA6BDA0EA96FAC6BDE0E97
:10153000AB6FAE6BE30EAD6FB06BE80EAF6FB26B1F
:10154000ED0EB16FB46BF20EB36FB66BF70EB56FF5
:10155000B86BFC0EB76F010EBA6FB96FBC6F050E9A
:10156000BB6F010EBE6F0A0EBD6F010EC06F0F0E76
:10157000BF6F010EC26F140EC16F010EC46F190E42
:10158000C36F010EC66F1E0EC56F010EC86F230E0E
:10159000C76F010ECA6F280EC96F010ECC6F2C0EDB
:1015A000CB6F010ECE6F310ECD6F010ED06F360EA8
:1015B000CF6F010ED26F3B0ED16F010ED46F400E74
:1015C000D36F010ED66F450ED56F010ED86F4A0E40
:1015D000D76F010EDA6F4F0ED96F010EDC6F530E0D
:1015E000DB6F010EDE6F580EDD6F010EE06F5D0EDA
:1015F000DF6F010EE26F620EE16F010EE46F670EA6
:10160000E36F010EE66F6C0EE56F010EE86F710E71
:10161000E76F010EEA6F760EE96F010EEC6F7A0E3E
:10162000EB6F010EEE6F7F0EED6F010EF06F840E0B
:10163000EF6F010EF26F890EF16F010EF46F8E0ED7
:10164000F36F010EF66F930EF56F010EF86F980EA3
:10165000F76F010EFA6F9D0EF96F010EFC6FA10E70
:10166000FB6F010EFE6FA60EFD6F010E0401006FF1
:10167000AB0E0301FF6F010E0401026FB00E016F8C
:10168000010E046FB50E036F010E066FBA0E056FE3
:10169000010E086FBF0E076F010E0A6FC40E096FAF
:1016A000010E0C6FC80E0B6F010E0E6FCD0E0D6F7D
:1016B000010E106FD20E0F6F010E126FD70E116F49
:1016C000010E146FDC0E136F010E166FE10E156F15
:1016D000010E186FE60E176F010E1A6FEB0E196FE1
:1016E000010E1C6FEF0E1B6F010E1E6FF40E1D6FAF
:1016F000010E206FF90E1F6F010E226FFE0E216F7B
:10170000020E246F030E236F020E266F080E256F44
:10171000020E286F0D0E276F020E2A6F120E296F10
:10172000020E2C6F160E2B6F020E2E6F1B0E2D6FDE
:10173000020E306F200E2F6F020E326F250E316FAA
:10174000020E346F2A0E336F020E366F2F0E356F76
:10175000020E386F340E376F020E3A6F390E396F42
:10176000020E3C6F3D0E3B6F020E3E6F420E3D6F10
:10177000020E406F470E3F6F020E426F4C0E416FDC
:10178000020E446F510E436F020E466F560E456FA8
:10179000020E486F5B0E476F020E4A6F600E496F74
:1017A000020E4C6F640E4B6F020E4E6F690E4D6F42
:1017B000020E506F6E0E4F6F020E526F730E516F0E
:1017C000020E546F780E536F020E566F7D0E556FDA
:1017D000020E586F820E576F020E5A6F870E596FA6
:1017E000020E5C6F8B0E5B6F020E5E6F900E5D6F74
:1017F000020E606F950E5F6F646B2F0E636F666BEA
:10180000340E656F686B390E676F6A6B3E0E696FD9
:101810006C6B420E6B6F6E6B470E6D6F706B4C0E88
:101820006F6F726B510E716F746B560E736F766BB8
:101830005B0E756F786B600E776F7A6B650E796FE4
:101840007C6B690E7B6F7E6B6E0E7D6F806B730E93
:101850007F6F826B780E816F846B7D0E836F866BDA
:10186000820E856F886B870E876F8A6B8C0E896FEF
:101870008C6B900E8B6F8E6B950E8D6F906B9A0E9E
:101880008F6F926B9F0E916F946BA40E936F966BFC
:10189000A90E956F986BAE0E976F9A6BB30E996FFA
:1018A0009C6BB70E9B6F9E6BBC0E9D6FA06BC10EA9
:1018B0009F6FA26BC60EA16FA46BCB0EA36FA66B1E
:1018C000D00EA56FA86BD50EA76FAA6BDA0EA96F05
:1018D000AC6BDE0EAB6FAE6BE30EAD6FB06BE80EB4
:1018E000AF6FB26BED0EB16FB46BF20EB36FB66B40
:1018F000F70EB56FB86BFC0EB76F010EBA6FB96F0C
:10190000BC6F050EBB6F010EBE6F0A0EBD6F010EE0
:10191000C06F0F0EBF6F010EC26F140EC16F010EAC
:10192000C46F190EC36F010EC66F1E0EC56F010E78
:10193000C86F230EC76F010ECA6F280EC96F010E44
:10194000CC6F2C0ECB6F010ECE6F310ECD6F010E12
:10195000D06F360ECF6F010ED26F3B0ED16F010EDE
:10196000D46F400ED36F010ED66F450ED56F010EAA
:10197000D86F4A0ED76F010EDA6F4F0ED96F010E76
:10198000DC6F530EDB6F010EDE6F580EDD6F010E44
:10199000E06F5D0EDF6F010EE26F620EE16F010E10
:1019A000E46F670EE36F010EE66F6C0EE56F010EDC
:1019B000E86F710EE76F010EEA6F760EE96F010EA8
:1019C000EC6F7A0EEB6F010EEE6F7F0EED6F010E76
:1019D000F06F840EEF6F010EF26F890EF16F010E42
:1019E000F46F8E0EF36F010EF66F930EF56F010E0E
:1019F000F86F980EF76F010EFA6F9D0EF96F010EDA
:101A0000FC6FA10EFB6F010EFE6FA60EFD6F010EA7
:101A10000501006FAB0E0401FF6F010E0501026F9F
:101A2000B00E016F010E046FB50E036F010E066F4D
:101A3000BA0E056F010E086FBF0E076F010E0A6F19
:101A4000C40E096F010E0C6FC80E0B6F010E0E6FE6
:101A5000CD0E0D6F010E106FD20E0F6F010E126FB3
:101A6000D70E116F010E146FDC0E136F010E166F7F
:101A7000E10E156F010E186FE60E176F010E1A6F4B
:101A8000EB0E196F010E1C6FEF0E1B6F010E1E6F18
:101A9000F40E1D6F010E206FF90E1F6F010E226FE5
:101AA000FE0E216F020E246F030E236F020E266FAF
:101AB000080E256F020E286F0D0E276F020E2A6F7B
:101AC000120E296F020E2C6F160E2B6F020E2E6F48
:101AD0001B0E2D6F020E306F200E2F6F020E326F15
:101AE000250E316F020E346F2A0E336F020E366FE1
:101AF0002F0E356F020E386F340E376F020E3A6FAD
:101B0000390E396F020E3C6F3D0E3B6F020E3E6F79
:101B1000420E3D6F020E406F470E3F6F020E426F46
:101B20004C0E416F020E446F510E436F020E466F12
:101B3000560E456F020E486F5B0E476F020E4A6FDE
:101B4000600E496F020E4C6F640E4B6F020E4E6FAB
:101B5000690E4D6F020E506F6E0E4F6F020E526F78
:101B6000730E516F020E546F780E536F020E566F44
:101B70007D0E556F020E586F820E576F020E5A6F10
:101B8000870E596F020E5C6F8B0E5B6F020E5E6FDD
:101B9000900E5D6F020E606F950E5F6F646B510E5D
:101BA000636F666B530E656F686B550E676F6A6B7C
:101BB000570E696F6C6B580E6B6F6E6B5A0E6D6FB4
:101BC000706B5C0E6F6F726B5E0E716F746B600E7C
:101BD000736F766B610E756F786B630E776F7A6BD0
:101BE000650E796F7C6B670E7B6F7E6B680E7D6F09
:101BF000806B6A0E7F6F826B6C0E816F846B6E0ED2
:101C0000836F866B700E856F886B710E876F8A6B22
:101C1000730E896F8C6B750E8B6F8E6B770E8D6F5D
:101C2000906B780E8F6F926B7A0E916F946B7C0E27
:101C3000936F966B7E0E956F986B800E976F9A6B75
:101C4000810E996F9C6B830E9B6F9E6B850E9D6FB3
:101C5000A06B870E9F6FA26B880EA16FA46B8A0E7C
:101C6000A36FA66B8C0EA56FA86B8E0EA76FAA6BC9
:101C7000900EA96FAC6B910EAB6FAE6B930EAD6F08
:101C8000B06B950EAF6FB26B970EB16FB46B980ED1
:101C9000B36FB66B9A0EB56FB86B9C0EB76FBA6B1D
:101CA0009E0EB96FBC6BA00EBB6FBE6BA10EBD6F5D
:101CB000C06BA30EBF6FC26BA50EC16FC46BA70E26
:101CC000C36FC66BA90EC56FC86BAA0EC76FCA6B70
:101CD000AC0EC96FCC6BAE0ECB6FCE6BB00ECD6FB2
:101CE000D06BB10ECF6FD26BB30ED16FD46BB50E7C
:101CF000D36FD66BB70ED56FD86BB90ED76FDA6BC3
:101D0000BA0ED96FDC6BBC0EDB6FDE6BBE0EDD6F07
:101D1000E06BC00EDF6FE26BC10EE16FE46BC30ED0
:101D2000E36FE66BC50EE56FE86BC70EE76FEA6B16
:101D3000C90EE96FEC6BCA0EEB6FEE6BCC0EED6F5C
:101D4000F06BCE0EEF6FF26BD00EF16FF46BD10E25
:101D5000F36FF66BD30EF56FF86BD50EF76FFA6B6A
:101D6000D70EF96FFC6BD90EFB6FFE6BDA0EFD6FB1
:101D70000601006BDC0E0501FF6F0601026BDE0E33
:101D8000016F046BE00E036F066BE10E056F086BCD
:101D9000E30E076F0A6BE50E096F0C6BE70E0B6F16
:101DA0000E6BE90E0D6F106BEA0E0F6F126BEC0EDF
:101DB000116F146BEE0E136F166BF00E156F186B20
:101DC000F10E176F1A6BF30E196F1C6BF50E1B6F6C
:101DD0001E6BF70E1D6F206BF90E1F6F226BFA0E34
:101DE000216F246BFC0E236F266BFE0E256F010EF8
:101DF000286F276B2A6F296F2C6F030E2B6F010E34
:101E00002E6F050E2D6F010E306F070E2F6F010E16
:101E1000326F090E316F010E346F0A0E336F010EEF
:101E2000366F0C0E356F010E386F0E0E376F010EC8
:101E30003A6F100E396F010E3C6F120E3B6F010EA0
:101E40003E6F130E3D6F010E406F150E3F6F010E7A
:101E5000426F170E416F010E446F190E436F010E52
:101E6000466F1A0E456F010E486F1C0E476F010E2C
:101E70004A6F1E0E496F010E4C6F200E4B6F010E04
:101E80004E6F220E4D6F010E506F230E4F6F010EDD
:101E9000526F250E516F010E546F270E536F010EB6
:101EA000566F290E556F010E586F2A0E576F010E8F
:101EB0005A6F2C0E596F010E5C6F2E0E5B6F010E68
:101EC0005E6F300E5D6F010E606F320E5F6F646B80
:101ED0002F0E636F666B340E656F686B390E676F1C
:101EE0006A6B3E0E696F6C6B420E6B6F6E6B470ECA
:101EF0006D6F706B4C0E6F6F726B510E716F746BF8
:101F0000560E736F766B5B0E756F786B600E776F26
:101F10007A6B650E796F7C6B690E7B6F7E6B6E0ED4
:101F20007D6F806B730E7F6F826B780E816F846B19
:101F30007D0E836F866B820E856F886B870E876F31
:101F40008A6B8C0E896F8C6B900E8B6F8E6B950EDF
:101F50008D6F906B9A0E8F6F926B9F0E916F946B3B
:101F6000A40E936F966BA90E956F986BAE0E976F3C
:101F70009A6BB30E996F9C6BB70E9B6F9E6BBC0EEA
:101F80009D6FA06BC10E9F6FA26BC60EA16FA46B5D
:101F9000CB0EA36FA66BD00EA56FA86BD50EA76F47
:101FA000AA6BDA0EA96FAC6BDE0EAB6FAE6BE30EF5
:101FB000AD6FB06BE80EAF6FB26BED0EB16FB46B7F
:101FC000F20EB36FB66BF70EB56FB86BFC0EB76F52
:101FD000010EBA6FB96FBC6F050EBB6F010EBE6FFD
:101FE0000A0EBD6F010EC06F0F0EBF6F010EC26FE4
:101FF000140EC16F010EC46F190EC36F010EC66FB0
:102000001E0EC56F010EC86F230EC76F010ECA6F7B
:10201000280EC96F010ECC6F2C0ECB6F010ECE6F48
:10202000310ECD6F010ED06F360ECF6F010ED26F15
:102030003B0ED16F010ED46F400ED36F010ED66FE1
:10204000450ED56F010ED86F4A0ED76F010EDA6FAD
:102050004F0ED96F010EDC6F530EDB6F010EDE6F7A
:10206000580EDD6F010EE06F5D0EDF6F010EE26F47
:10207000620EE16F010EE46F670EE36F010EE66F13
:102080006C0EE56F010EE86F710EE76F010EEA6FDF
:10209000760EE96F010EEC6F7A0EEB6F010EEE6FAC
:1020A0007F0EED6F010EF06F840EEF6F010EF26F79
:1020B000890EF16F010EF46F8E0EF36F010EF66F45
:1020C000930EF56F010EF86F980EF76F010EFA6F11
:1020D0009D0EF96F010EFC6FA10EFB6F010EFE6FDE
:1020E000A60EFD6F010E0701006FAB0E0601FF6F1C
:1020F000010E0701026FB00E016F010E046FB50EE5
:10210000036F010E066FBA0E056F010E086FBF0E4A
:10211000076F010E0A6FC40E096F010E0C6FC80E17
:102120000B6F010E0E6FCD0E0D6F010E106FD20EE4
:102130000F6F010E126FD70E116F010E146FDC0EB0
:10214000136F010E166FE10E156F010E186FE60E7C
:10215000176F010E1A6FEB0E196F010E1C6FEF0E49
:102160001B6F010E1E6FF40E1D6F010E206FF90E16
:102170001F6F010E226FFE0E216F020E246F030EE1
:10218000236F020E266F080E256F020E286F0D0EAC
:10219000276F020E2A6F120E296F020E2C6F160E79
:1021A0002B6F020E2E6F1B0E2D6F020E306F200E46
:1021B0002F6F020E326F250E316F020E346F2A0E12
:1021C000336F020E366F2F0E356F020E386F340EDE
:1021D000376F020E3A6F390E396F020E3C6F3D0EAB
:1021E0003B6F020E3E6F420E3D6F020E406F470E78
:1021F0003F6F020E426F4C0E416F020E446F510E44
:10220000436F020E466F560E456F020E486F5B0E0F
:10221000476F020E4A6F600E496F020E4C6F640EDC
:102220004B6F020E4E6F690E4D6F020E506F6E0EA9
:102230004F6F020E526F730E516F020E546F780E75
:10224000536F020E566F7D0E556F020E586F820E41
:10225000576F020E5A6F870E596F020E5C6F8B0E0E
:102260005B6F020E5E6F900E5D6F020E606F950EDB
:082270005F6F00011200FFD7AF
:020000040030CA
:0300010006160ED2
:020005008580F4
:060008000FC00FE00F40E5
:00000001FF
